:020000040000FA
:020000001728BF
:080008008A0182073F3406342F
:100010005B344F3466346D347D3407347F346F3451
:1000200077347C3439345E34793471340800FF30ED
:10003000A200FF30A3002B210F21292107309F00B0
:1000400022107921A2107821221177212310742106
:10005000A310732123117221A31171212312702186
:10006000A3126F2123136E21A3136D21A601A701F3
:100070007B30A800FF30AB005520AB0B3C28323062
:10008000AB005520AB0B4128AB018B20A010201DED
:100090004A28A0142C08A9002D08AA002908A600A7
:1000A0002A08A70055203A2854282608AE000A300E
:1000B000AF008F213008AD002D08AC002608B0003D
:1000C0000A30B10080213208AF002F08AE002C08A2
:1000D0003321B0003008FF3A65212410642101303B
:1000E0003A21241464212E083321B0003008FF3A4D
:1000F0006521A410632101303A21A414632127084B
:100100003321B0003008FF3A65212411622101300B
:100110003A2124156229AD002B08483EB000AE20DC
:100120003108AE003208AF00AE1FA42820152E08FB
:10013000FF3AAC00AF1FA12801302C02AC00AD018A
:10014000A3280530AD00AD2820112E08AC00AF1F4C
:10015000AC280530AD00AD28AD010800B200300874
:10016000BA20C1203308B100DB20C1203308B2001F
:10017000DB200F29B3001C210310330D013ECE20DC
:10018000DD28B3000830B4000310B30DEB203310AA
:10019000A01DCB283314B40BC4280800B4000830C9
:1001A000B500A011B41FD528A015FE200310B40D72
:1001B000B50BD1280800A011FE282921221675218F
:1001C0002921A215762129218519E728E42829214A
:1001D000A211762129292921221675212921A2156A
:1001E000762129218519F528F2282921A011051E3B
:1001F000FA28A0152921A2117621292929212212C4
:10020000A01D0329221675212921A2157621292155
:1002100085190B2908292921A211762129292921AB
:10022000221275212921A21176212921A2157621D8
:1002300029212216752129292921221675212921F2
:10024000A21576212921221275212921A2117621B8
:1002500029290C305329A4116121A21176212412DD
:10026000602122127529B10031080F390420B20033
:1002700032080800B1003108B2000A30B300013082
:100280004129B400FF30B5003308B7003208B6008A
:100290001730350703184929B60B4829B70B4629EB
:1002A000B40B44290800B600F430B700FC30B800A5
:1002B00036083707031C0034380703185C29080088
:1002C0006A296A296A296A296A29A50067292508ED
:1002D000860008002408850008007A297A297A29EE
:1002E0007A297A297A297A297A297D297D297D29ED
:1002F0007D297D2923086600080022086500080082
:10030000B10803198C2931083002031888298C2977
:1003100031083002B00083293008B2000800B10172
:10032000AF0803199D292F082E02031898299D292B
:100330002F082E02AE00B10A93293108B000080040
:02400E00103F61
:00000001FF
